:020000040000FA
:0A0000000000000045EF01F054D1AC
:08001800A0D10A6A096EFF0E77
:1000200009260A2200D0D8A01200030E086EE60EA0
:1000300002D8F5D7086AFE0F076EE86A085AD8A0FA
:1000400012000000070600D0F8D710500C5C156EA7
:1000500011E2156C0C5010C00CF0106E0D5011C058
:100060000DF0116E0E5012C00EF0126E0F5013C034
:100070000FF0136E1A0E156074D0105272E0146AED
:100080000D50176E1118186E0D8E118E080E155E1C
:1000900008E313C014F012C013F011C012F0116A7B
:1000A000F5D7152607E0D8901132123213321432E8
:1000B000152EF9D718AE33D013500F5E12500E5ACA
:1000C00011500D5A07E2D880000E0F560E560D56ED
:1000D000800E171A146C04E00F06000E0E5A0D5A0B
:1000E000040E156E0D660DD00EC00DF00FC00EF093
:1000F00014C00FF0146A080E0C5E29E3152EF2D717
:1001000026D00DBE08D0D89014360F360E360D36D8
:100110000C2EF7D71CD014AE22D0146A0FD0135077
:100120000F2612500E2211500D2206E30D320E3210
:100130000F3214320C4A0DD014AE11D00F3E0FD036
:100140000E3E0DD00D3E0BD0D8800F90EFD70C6A2D
:1001500002D016820C680F6A0E6A800E0D6E17AE02
:100160000D9E0F5012000CC017F00D500FC00DF077
:100170000F6E0F3617320F32166A0F36173602E33C
:100180001684167E06E11680176A0F6A0E6A0D6ADB
:100190000BD0172803E0D8800F3206D0D8900F324A
:1001A00002E1168201D0168616B604D016A20FD030
:1001B00016B407D07F0E0F6EFF0E0E6E0D6E0C6E16
:1001C00023D0800E0F6E01D00F6A000EF6D716B046
:1001D000FBD70C6A9F0E1760EBD77E0E1764F4D71F
:1001E0009E0E175C07E0D8900F320E320D320C32A3
:1001F000172AF6D716A408D0D880000E0C560D5634
:100200000E560F560FAEE0D70C5012000E6A0F6A52
:10021000189E0AD0189E0FAE07D0D880000E0C563C
:100220000D560E560F56188E960E176E0F5209E089
:10023000080E17260DC00CF00EC00DF00FC00EF00A
:1002400011D00E520FE1080E175E0D5007E1080E97
:10025000175E0C5002E10F5010D00C6A0E6E0CC0ED
:100260000DF00C6A0EBE06D0D8900C360D360E3648
:100270001706F8D718AE0E9E17500CC00FF00C6E74
:100280000E500DC00EF00D6E1200400E166E4F0E89
:10029000AF6E240EAC6E900EAB6E00010F0EC16EF1
:1002A000070EB46EC69A400E926E936AC00E946E9C
:1002B0006BD0F2A402D0F29411009EAA19D0060EBF
:1002C000AB1412E1E2CF75F0E1CF74F0762A10EEB4
:1002D000BEF07650E126000EE222AECFE7FF75C0F9
:1002E000E2FF74C0E1FF1100AE50AE50AB98AB8896
:1002F00011007650775C14E0772AEACF08F0E9CF56
:1003000007F000EEBEF07750E926000EEA22EF502B
:10031000076E08C0EAFF07C0E9FFD880120004D0CA
:10032000E868076ED8A012001200766A776A9D8A84
:100330009F8AF28EF28C12009D9A00EEBEF0010EA2
:10034000F46EF36AF306000EF45AEE6AF450F310FA
:10035000F9E1766A776A9D8A1200F29EE0CFBEF3D9
:10036000D8CFBFF3E8CFC0F3F28E0001A192F29E86
:10037000BEC3E0FFBFC3D8FFC0C3E8FFF28E1000CA
:100380009EA8FED7AD6E12000A0E47DE92928992A9
:1003900092968996929A899A939C8A9C93988A9825
:1003A00093948A9493908A9094988B9894928B9239
:1003B00094968B9692948994929089909298899829
:1003C000939E8A9E939A8A9A93968A9693928A92F9
:1003D000949A8B9A94908B9094948B94546A536AC9
:1003E0004E6A4D6A506A4F6A526A516A00EE96F040
:1003F000280EEE68E82EFDD78C6B8D6B8E6B8F6BA5
:10040000906B916B926B936B946B956B796A786A36
:100410007B6A7A6A7D6A7C6A7F6A7E6A816B806B9E
:10042000836B826B856B846B876B866B896B886B48
:100430008B6B8A6B566A556A586A576A5A6A596A48
:100440005C6A5B6A5E6A5D6A606A5F6A626A616A68
:10045000646A636A666A656A686A676A66DF6CDF2F
:10046000CD6AF294F28A870ED56EB16AA192A0820B
:10047000D08EA292B10EB16E24EC0DF024EC0FF0F0
:100480006D2AE86A6DB2010F6EB0010806E16E7068
:10049000692A000E6A226B226C222BDF196EC10EB4
:1004A000195C06E3FE0E195C01E21B6A0CEF06F014
:1004B00019AE29D01B6A800E195C05E119C01BF02A
:1004C0001C681D681ED0900E195C05E119C01BF058
:1004D0001E681F6816D0A00E195C05E119C01BF03C
:1004E000206821680ED0B00E195C05E119C01BF020
:1004F0002268236806D0C00E195C03E119C01BF006
:1005000024680AEF06F01B5204E10CEF06F00AEF34
:1005100006F0800E1B5CD8A499D01C2803E119C0FA
:100520001CF090D019C01DF0330E1C5C0BE14D90F7
:1005300053904F90519099699869976996698992FB
:1005400089947DD0340E1C5C0BE14D924F925192F8
:1005500053929D699C699B699A69899689906FD02D
:10056000350E1C5C0BE14D944F9451945394A1694A
:10057000A0699F699E69899A899861D0360E1C5C32
:100580000BE14D964F9651965396A569A469A369C0
:10059000A2698A9C8A9E53D0370E1C5C0BE14D9851
:1005A0004F9851985398A969A869A769A6698A982C
:1005B0008A9A45D0380E1C5C0BE14D9A4F9A519A9D
:1005C000539AAD69AC69AB69AA698A948A9637D0A7
:1005D000390E1C5C0BE14D9C4F9C519C539CB169A6
:1005E000B069AF69AE698A908A9229D03A0E1C5CD4
:1005F0000BE14D9E4F9E519E539EB569B469B36900
:10060000B2698B988B9A1BD03B0E1C5C0BE14E9011
:10061000509052905490B969B869B769B6698B9295
:100620008B900DD03C0E1C5C0AE14E92509252927F
:100630005492BD69BC69BB69BA698B968B941C687E
:100640000AEF06F00CEF06F00AEF06F0900E1B5CC6
:10065000D8A4E2EF05F01E2804E119C01EF0E0EF77
:1006600005F019C01FF01F52D8A494D0330E1E5CA1
:100670000BE14D904F90519053909969986997690B
:1006800096698992899481D0340E1E5C0BE14D925B
:100690004F92519253929D699C699B699A69899680
:1006A000899073D0350E1E5C0BE14D944F9451949C
:1006B0005394A169A0699F699E69899A899865D0B8
:1006C000360E1E5C0BE14D964F9651965396A569DA
:1006D000A469A369A2698A9C8A9E57D0370E1E5CC2
:1006E0000BE14D984F9851985398A969A869A7694B
:1006F000A6698A988A9A49D0380E1E5C0BE14D9AF9
:100700004F9A519A539AAD69AC69AB69AA698A94B8
:100710008A963BD0390E1E5C0BE14D9C4F9C519C40
:10072000539CB169B069AF69AE698A908A922DD045
:100730003A0E1E5C0BE14D9E4F9E519E539EB56935
:10074000B469B369B2698B988B9A1FD03B0E1E5C5B
:100750000BE14E90509052905490B969B869B769C6
:10076000B6698B928B9011D03C0E1E5C0BE14E92C1
:10077000509252925492BD69BC69BB69BA698B961A
:100780008B9403D01E680CEF06F01E680AEF06F08B
:10079000E0EF05F0330E1E5C32E14D8001EEBEF05D
:1007A000D8901F34E926000EEA22EECF55F0EFCFA5
:1007B00056F055506924006E56506A20016E000EA6
:1007C0006B20026E000E6C20036E03C099F002C015
:1007D00098F001C097F000C096F089828C530DE02C
:1007E000538002EEBEF0D8908C35E926000EEA2246
:1007F000EECF78F0EFCF79F001D05390DFD1340E07
:100800001E5C32E14D8201EEBEF0D8901F34E92625
:10081000000EEA22EECF57F0EFCF58F05750692480
:10082000006E58506A20016E000E6B20026E000EA2
:100830006C20036E03C09DF002C09CF001C09BF0D1
:1008400000C09AF089868D530DE0538202EEBEF00F
:10085000D8908D35E926000EEA22EECF7AF0EFCF60
:100860007BF001D05392AAD1350E1E5C32E14D844B
:1008700001EEBEF0D8901F34E926000EEA22EECF3A
:1008800059F0EFCF5AF059506924006E5A506A203F
:10089000016E000E6B20026E000E6C20036E03C012
:1008A000A1F002C0A0F001C09FF000C09EF0898AB4
:1008B0008E530DE0538402EEBEF0D8908E35E926BB
:1008C000000EEA22EECF7CF0EFCF7DF001D0539402
:1008D00075D1360E1E5C32E14D8601EEBEF0D89029
:1008E0001F34E926000EEA22EECF5BF0EFCF5CF07A
:1008F0005B506924006E5C506A20016E000E6B2014
:10090000026E000E6C20036E03C0A5F002C0A4F0BE
:1009100001C0A3F000C0A2F08A8C8F530DE0538673
:1009200002EEBEF0D8908F35E926000EEA22EECF17
:100930007EF0EFCF7FF001D0539640D1370E1E5C92
:1009400032E14D8801EEBEF0D8901F34E926000E4A
:10095000EA22EECF5DF0EFCF5EF05D506924006ECD
:100960005E506A20016E000E6B20026E000E6C203D
:10097000036E03C0A9F002C0A8F001C0A7F000C038
:10098000A6F08A8890530DE0538802EEBEF0D8900E
:100990009035E926000EEA22EECF80F0EFCF81F00D
:1009A00001D053980BD1380E1E5C32E14D8A01EE16
:1009B000BEF0D8901F34E926000EEA22EECF5FF099
:1009C000EFCF60F05F506924006E60506A20016EC6
:1009D000000E6B20026E000E6C20036E03C0ADF0A3
:1009E00002C0ACF001C0ABF000C0AAF08A84915301
:1009F0000DE0538A02EEBEF0D8909135E926000E44
:100A0000EA22EECF82F0EFCF83F001D0539AD6D016
:100A1000390E1E5C32E14D8C01EEBEF0D8901F34D1
:100A2000E926000EEA22EECF61F0EFCF62F06150CE
:100A30006924006E62506A20016E000E6B20026E07
:100A4000000E6C20036E03C0B1F002C0B0F001C014
:100A5000AFF000C0AEF08A8092530DE0538C02EEEE
:100A6000BEF0D8909235E926000EEA22EECF84F04F
:100A7000EFCF85F001D0539CA1D03A0E1E5C32E13D
:100A80004D8E01EEBEF0D8901F34E926000EEA220A
:100A9000EECF63F0EFCF64F063506924006E6450D2
:100AA0006A20016E000E6B20026E000E6C20036E39
:100AB00003C0B5F002C0B4F001C0B3F000C0B2F0A2
:100AC0008B8893530DE0538E02EEBEF0D890933591
:100AD000E926000EEA22EECF86F0EFCF87F001D0B4
:100AE000539E6CD03B0E1E5C32E14E8001EEBEF098
:100AF000D8901F34E926000EEA22EECF65F0EFCF42
:100B000066F065506924006E66506A20016E000E22
:100B10006B20026E000E6C20036E03C0B9F002C0A1
:100B2000B8F001C0B7F000C0B6F08B8294530DE06E
:100B3000548002EEBEF0D8909435E926000EEA22E9
:100B4000EECF88F0EFCF89F001D0549037D03C0E33
:100B50001E5C32E14E8201EEBEF0D8901F34E926D1
:100B6000000EEA22EECF67F0EFCF68F067506924FD
:100B7000006E68506A20016E000E6B20026E000E3F
:100B80006C20036E03C0BDF002C0BCF001C0BBF01E
:100B900000C0BAF08B8695530DE0548202EEBEF091
:100BA000D8909535E926000EEA22EECF8AF0EFCFF5
:100BB0008BF001D0549202D01E682ED01E682AD02D
:100BC0002BD028D0A00E1B5C0BE1202803E119C01C
:100BD00020F004D019C021F087EC0AF01DD01AD003
:100BE000B00E1B5C0BE1222803E119C022F004D0F7
:100BF00019C023F0E6EC0BF00FD00CD0C00E1B5C3C
:100C000008E1242804E119C024F0D2EC0BF004D050
:100C100001D002D04DEC0AF00A0E735CD8B045EF5B
:100C20000AF06F50695C70506A5871506B5872507E
:100C30006C58D8A030EF0AF0728E7352D8A465D0E9
:100C400053B008D0899289844D90996998699769C1
:100C5000966959D051A018D04D8055506924006E26
:100C600056506A20016E000E6B20026E000E6C2042
:100C7000036E03C099F002C098F001C097F000C065
:100C800096F0898251903FD04FA023D0899402EEF4
:100C9000BEF0D8908C35E926000EEA22EECF04F0A3
:100CA000EFCF05F004506924006E05506A20016EF4
:100CB000000E6B20026E000E6C20036E03C099F0D4
:100CC00002C098F001C097F000C096F04F9051809C
:100CD0001AD04DA018D0899278506924006E7950AE
:100CE0006A20016E000E6B20026E000E6C20036EF7
:100CF00003C099F002C098F001C097F000C096F0D0
:100D000089844F804D902FEF0AF0010E735CD8A4B8
:100D100065D053B208D0899689804D929D699C69AF
:100D20009B699A6959D051A218D04D8257506924B5
:100D3000006E58506A20016E000E6B20026E000E8D
:100D40006C20036E03C09DF002C09CF001C09BF0BC
:100D500000C09AF0898651923FD04FA223D089904B
:100D600002EEBEF0D8908D35E926000EEA22EECFD5
:100D700004F0EFCF05F004506924006E05506A209E
:100D8000016E000E6B20026E000E6C20036E03C01D
:100D90009DF002C09CF001C09BF000C09AF04F9201
:100DA00051821AD04DA218D089967A506924006ECB
:100DB0007B506A20016E000E6B20026E000E6C20CC
:100DC000036E03C09DF002C09CF001C09BF000C008
:100DD0009AF089804F824D922FEF0AF0020E735CD9
:100DE000D8A465D053B408D0899A89884D94A16954
:100DF000A0699F699E6959D051A418D04D8459505B
:100E00006924006E5A506A20016E000E6B20026E3B
:100E1000000E6C20036E03C0A1F002C0A0F001C060
:100E20009FF000C09EF0898A51943FD04FA423D0F8
:100E3000899802EEBEF0D8908E35E926000EEA229F
:100E4000EECF04F0EFCF05F004506924006E05509A
:100E50006A20016E000E6B20026E000E6C20036E85
:100E600003C0A1F002C0A0F001C09FF000C09EF03E
:100E70004F9451841AD04DA418D0899A7C5069247B
:100E8000006E7D506A20016E000E6B20026E000E17
:100E90006C20036E03C0A1F002C0A0F001C09FF05F
:100EA00000C09EF089884F844D942FEF0AF0030E06
:100EB000735CD8A465D053B608D08A9C8A8E4D96B0
:100EC000A569A469A369A26959D051A618D04D8615
:100ED0005B506924006E5C506A20016E000E6B202E
:100EE000026E000E6C20036E03C0A5F002C0A4F0D9
:100EF00001C0A3F000C0A2F08A8C51963FD04FA64B
:100F000023D08A9E02EEBEF0D8908F35E926000EDF
:100F1000EA22EECF04F0EFCF05F004506924006E12
:100F200005506A20016E000E6B20026E000E6C20D0
:100F3000036E03C0A5F002C0A4F001C0A3F000C07E
:100F4000A2F04F9651861AD04DA618D08A9C7E509A
:100F50006924006E7F506A20016E000E6B20026EC5
:100F6000000E6C20036E03C0A5F002C0A4F001C007
:100F7000A3F000C0A2F08A8E4F864D962FEF0AF0A4
:100F8000040E735CD8A464D053B808D08A988A8AB7
:100F90004D98A969A869A769A66959D051A818D020
:100FA0004D885D506924006E5E506A20016E000E0F
:100FB0006B20026E000E6C20036E03C0A9F002C00D
:100FC000A8F001C0A7F000C0A6F08A8851983FD0D1
:100FD0004FA823D08A9A02EEBEF0D8909035E92629
:100FE000000EEA22EECF04F0EFCF05F004506924A2
:100FF000006E05506A20016E000E6B20026E000E1E
:101000006C20036E03C0A9F002C0A8F001C0A7F0D5
:1010100000C0A6F04F9851881AD04DA818D08A98D1
:1010200080516924006E81516A20016E000E6B2090
:10103000026E000E6C20036E03C0A9F002C0A8F07F
:1010400001C0A7F000C0A6F08A8A4F884D9807D249
:10105000050E735CD8A464D053BA08D08A948A86EB
:101060004D9AAD69AC69AB69AA6959D051AA18D03B
:101070004D8A5F506924006E60506A20016E000E38
:101080006B20026E000E6C20036E03C0ADF002C038
:10109000ACF001C0ABF000C0AAF08A84519A3FD0F6
:1010A0004FAA23D08A9602EEBEF0D8909135E92659
:1010B000000EEA22EECF04F0EFCF05F004506924D1
:1010C000006E05506A20016E000E6B20026E000E4D
:1010D0006C20036E03C0ADF002C0ACF001C0ABF0F9
:1010E00000C0AAF04F9A518A1AD04DAA18D08A94FB
:1010F00082516924006E83516A20016E000E6B20BC
:10110000026E000E6C20036E03C0ADF002C0ACF0A6
:1011100001C0ABF000C0AAF08A864F8A4D9A9FD1D9
:10112000060E735CD8A464D053BC08D08A908A821F
:101130004D9CB169B069AF69AE6959D051AC18D056
:101140004D8C61506924006E62506A20016E000E61
:101150006B20026E000E6C20036E03C0B1F002C063
:10116000B0F001C0AFF000C0AEF08A80519C3FD01B
:101170004FAC23D08A9202EEBEF0D8909235E92689
:10118000000EEA22EECF04F0EFCF05F00450692400
:10119000006E05506A20016E000E6B20026E000E7C
:1011A0006C20036E03C0B1F002C0B0F001C0AFF01C
:1011B00000C0AEF04F9C518C1AD04DAC18D08A9024
:1011C00084516924006E85516A20016E000E6B20E7
:1011D000026E000E6C20036E03C0B1F002C0B0F0CE
:1011E00001C0AFF000C0AEF08A824F8C4D9C37D169
:1011F000070E735CD8A464D053BE08D08B988B8A3A
:101200004D9EB569B469B369B26959D051AE18D071
:101210004D8E63506924006E64506A20016E000E8A
:101220006B20026E000E6C20036E03C0B5F002C08E
:10123000B4F001C0B3F000C0B2F08B88519E3FD033
:101240004FAE23D08B9A02EEBEF0D8909335E926AC
:10125000000EEA22EECF04F0EFCF05F0045069242F
:10126000006E05506A20016E000E6B20026E000EAB
:101270006C20036E03C0B5F002C0B4F001C0B3F03F
:1012800000C0B2F04F9E518E1AD04DAE18D08B9840
:1012900086516924006E87516A20016E000E6B2012
:1012A000026E000E6C20036E03C0B5F002C0B4F0F5
:1012B00001C0B3F000C0B2F08B8A4F8E4D9ECFD0EC
:1012C000080E735CD8A464D054B008D08B928B8085
:1012D0004E90B969B869B769B66959D052A018D0AB
:1012E0004E8065506924006E66506A20016E000EC3
:1012F0006B20026E000E6C20036E03C0B9F002C0BA
:10130000B8F001C0B7F000C0B6F08B8252903FD069
:1013100050A023D08B9002EEBEF0D8909435E926F1
:10132000000EEA22EECF04F0EFCF05F0045069245E
:10133000006E05506A20016E000E6B20026E000EDA
:101340006C20036E03C0B9F002C0B8F001C0B7F062
:1013500000C0B6F0509052801AD04EA018D08B9298
:1013600088516924006E89516A20016E000E6B203D
:10137000026E000E6C20036E03C0B9F002C0B8F01C
:1013800001C0B7F000C0B6F08B8050804E9067D09F
:10139000090E735CD8A463D054B208D08B968B84AA
:1013A0004E92BD69BC69BB69BA6959D052A218D0C6
:1013B0004E8267506924006E68506A20016E000EEC
:1013C0006B20026E000E6C20036E03C0BDF002C0E5
:1013D000BCF001C0BBF000C0BAF08B8652923FD087
:1013E00050A223D08B9402EEBEF0D8909535E9261A
:1013F000000EEA22EECF04F0EFCF05F0045069248E
:10140000006E05506A20016E000E6B20026E000E09
:101410006C20036E03C0BDF002C0BCF001C0BBF085
:1014200000C0BAF0509252821AD04EA218D08B96B9
:101430008A516924006E8B516A20016E000E6B2068
:10144000026E000E6C20036E03C0BDF002C0BCF043
:1014500001C0BBF000C0BAF08B8450824E921DD800
:101460006CAE12D06C6A6B6A6A6A696A4E6A4D6ABF
:10147000506A4F6A526A516A546A536A00EE96F093
:10148000280EEE68E82EFDD706D06CAE04D06C6A4C
:101490006B6A6A6A696A40EF02F07368728E1A6A50
:1014A0000A0E1A5C33E2D8901A34E96EEA6AEA3618
:1014B000E936EA36960EE926000EEA22EFCF00F072
:1014C000ECCF01F0ECCF02F0ECCF03F06F50005CFA
:1014D00070500158715002587250035815E2D8905C
:1014E0001A34E96EEA6AEA36E936EA36960EE926F1
:1014F000000EEA22EFCF6FF0ECCF70F0ECCF71F07E
:10150000ECCF72F01AC073F01A2ACAE31200330E3D
:10151000205C1EE121C08CF08C530CE002EEBEF08A
:10152000D8908C35E926000EEA22EECF78F0EFCF86
:1015300079F00DD0796A786A53904D904F90519020
:10154000996998699769966989948992A6DF28D1E3
:10155000340E205C1EE121C08DF08D530CE002EEB4
:10156000BEF0D8908D35E926000EEA22EECF7AF053
:10157000EFCF7BF00DD07B6A7A6A53924D924F92F7
:1015800051929D699C699B699A698990899685DFCA
:1015900007D1350E205C1EE121C08EF08E530CE089
:1015A00002EEBEF0D8908E35E926000EEA22EECF8C
:1015B0007CF0EFCF7DF00DD07D6A7C6A53944D9422
:1015C0004F945194A169A0699F699E698998899AED
:1015D00064DFE6D0360E205C1EE121C08FF08F5311
:1015E0000CE002EEBEF0D8908F35E926000EEA221C
:1015F000EECF7EF0EFCF7FF00DD07F6A7E6A5396FC
:101600004D964F965196A569A469A369A2698A9ED1
:101610008A9C43DFC5D0370E205C1EE121C090F0CC
:1016200090530CE002EEBEF0D8909035E926000E03
:10163000EA22EECF80F0EFCF81F00DD0816B806B8E
:1016400053984D984F985198A969A869A769A669B8
:101650008A9A8A9822DFA4D0380E205C1EE121C02D
:1016600091F091530CE002EEBEF0D8909135E9264E
:10167000000EEA22EECF82F0EFCF83F00DD0836B25
:10168000826B539A4D9A4F9A519AAD69AC69AB6986
:10169000AA698A968A9401DF83D0390E205C1EE104
:1016A00021C092F092530CE002EEBEF0D890923539
:1016B000E926000EEA22EECF84F0EFCF85F00DD0C0
:1016C000856B846B539C4D9C4F9C519CB169B06958
:1016D000AF69AE698A928A90E0DE62D03A0E205CF1
:1016E0001EE121C093F093530CE002EEBEF0D890BF
:1016F0009335E926000EEA22EECF86F0EFCF87F091
:101700000DD0876B866B539E4D9E4F9E519EB56943
:10171000B469B369B2698B9A8B98BFDE41D03B0E36
:10172000205C1EE121C094F094530CE002EEBEF068
:10173000D8909435E926000EEA22EECF88F0EFCF5C
:1017400089F00DD0896B886B54904E9050905290D8
:10175000B969B869B769B6698B908B929EDE20D063
:101760003C0E205C1DE121C095F095530CE002EE8B
:10177000BEF0D8909535E926000EEA22EECF8AF029
:10178000EFCF8BF00DD08B6B8A6B54924E925092B0
:101790005292BD69BC69BB69BA698B948B967DDE38
:1017A00020681200070E2416245203E124EC0FF0E7
:1017B0000BD0020E245C03E165EC0FF005D0030EA4
:1017C000245CD8B490EC0FF0246812001E0E225C4A
:1017D000D8A4C8D02352D8A442D0546A536A796A94
:1017E000786A8C6B7B6A7A6A8D6B7D6A7C6A8E6B99
:1017F0007F6A7E6A8F6B816B806B906B836B826B71
:10180000916B856B846B926B876B866B936B896B2B
:10181000886B946B8B6B8A6B956B4E6A4D6A506AC2
:101820004F6A526A516A00EE96F0280EEE68E82E72
:10183000FDD789928996899A8A9C8A988A948A90F7
:101840008B988B928B968994899089988A9E8A9A94
:101850008A968A928B9A8B908B941FDE82D023C0BB
:101860008CF002EEBEF0D8902334E926000EEA2276
:10187000EECF78F0EFCF79F023C08DF002EEBEF01E
:10188000D8902334E926000EEA22EECF7AF0EFCF8B
:101890007BF023C08EF002EEBEF0D8902334E92610
:1018A000000EEA22EECF7CF0EFCF7DF023C08FF068
:1018B00002EEBEF0D8902334E926000EEA22EECFE5
:1018C0007EF0EFCF7FF023C090F002EEBEF0D89014
:1018D0002334E926000EEA22EECF80F0EFCF81F02C
:1018E00023C091F002EEBEF0D8902334E926000E1A
:1018F000EA22EECF82F0EFCF83F023C092F002EE27
:10190000BEF0D8902334E926000EEA22EECF84F010
:10191000EFCF85F023C093F002EEBEF0D8902334D1
:10192000E926000EEA22EECF86F0EFCF87F023C043
:1019300094F002EEBEF0D8902334E926000EEA229D
:10194000EECF88F0EFCF89F023C095F002EEBEF025
:10195000D8902334E926000EEA22EECF8AF0EFCFAA
:101960008BF02ED0420E225C04E12352D8B42AD848
:1019700027D07B0E225C24E14E6A4D6A506A4F6A82
:10198000526A516A546A536A00EE96F0280EEE6865
:10199000E82EFDD789928996899A8A9C8A988A949A
:1019A0008A908B988B928B968994899089988A9E3D
:1019B0008A9A8A968A928B9A8B908B944DEC0AF035
:1019C000226812004E6A4D6A506A4F6A526A516A22
:1019D000546A536A00EE96F0280EEE68E82EFDD7A2
:1019E00089928996899A8A9C8A988A948A908B98F7
:1019F0008B928B968994899089988A9E8A9A8A96E6
:101A00008A928B9A8B908B94796A786A8C6B7B6ABA
:101A10007A6A8D6B7D6A7C6A8E6B7F6A7E6A8F6B59
:101A2000816B806B906B836B826B916B856B846B2E
:101A3000926B876B866B936B896B886B946B8B6BEC
:101A40008A6B956B4DEF0AF00201BF69BE695C0EAF
:101A5000C16F7A0EC06F590EC36F850EC26F580EDC
:101A6000C56F140EC46F560EC76FA90EC66F550E04
:101A7000C96F430EC86F530ECB6FE30ECA6F520E81
:101A8000CD6F890ECC6F510ECF6F350ECE6F4F0ECE
:101A9000D16FE60ED06F4E0ED36F9C0ED26F4D0EEF
:101AA000D56F580ED46F4C0ED76F190ED66F4A0EE5
:101AB000D96FDF0ED86F490EDB6FAA0EDA6F480EB2
:101AC000DD6F7A0EDC6F470EDF6F4F0EDE6F460E56
:101AD000E16F290EE06F450EE36F080EE26F430ED3
:101AE000E56FEB0EE46F420EE76FD30EE66F410E2B
:101AF000E96FBF0EE86F400EEB6FB00EEA6F3F0E5E
:101B0000ED6FA50EEC6F3E0EEF6F9E0EEE6F3D0E6D
:101B1000F16F9C0EF06F3C0EF36F9E0EF26F3B0E5A
:101B2000F56FA40EF46F3A0EF76FAE0EF66F390E26
:101B3000F96FBC0EF86F380EFB6FCE0EFA6F370ED2
:101B4000FD6FE30EFC6F360EFF6FFD0EFE6F360E5F
:101B50000301016F1A0E006F350E036F3B0E026F0B
:101B6000340E056F5F0E046F330E076F870E066F1E
:101B7000320E096FB20E086F310E0B6FE10E0A6F55
:101B8000310E0D6F140E0C6F300E0F6F490E0E6F6D
:101B90002F0E116F820E106F2E0E136FBE0E126F6E
:101BA0002D0E156FFD0E146F2D0E176F3F0E166F55
:101BB0002C0E196F850E186F2B0E1B6FCD0E1A6F22
:101BC0002B0E1D6F180E1C6F2A0E1F6F670E1E6FD7
:101BD000290E216FB80E206F290E236F0C0E226F75
:101BE000280E256F620E246F270E276FBC0E266FFE
:101BF000270E296F180E286F260E2B6F760E2A6F70
:101C0000250E2D6FD80E2C6F250E2F6F3C0E2E6FCC
:101C1000240E316FA20E306F240E336F0B0E326F15
:101C2000230E356F760E346F220E376FE40E366F4B
:101C3000220E396F540E386F210E3B6FC60E3A6F6D
:101C4000210E3D6F3B0E3C6F200E3F6FB20E3E6F7C
:101C5000200E416F2B0E406F1F0E436FA60E426F7A
:101C60001F0E456F240E446F1E0E476FA30E466F66
:101C70001E0E496F250E486F1D0E4B6FA90E4A6F41
:101C80001D0E4D6F2E0E4C6F1C0E4F6FB60E4E6F0D
:101C90001C0E516F3F0E506F1B0E536FCB0E526FC9
:101CA0001B0E556F580E546F1A0E576FE80E566F75
:101CB0001A0E596F790E586F1A0E5B6F0B0E5A6F12
:101CC000190E5D6FA00E5C6F190E5F6F360E5E6FA2
:101CD000180E616FCE0E606F180E636F680E626F24
:101CE000180E656F030E646F170E676FA00E666F98
:101CF000170E696F3F0E686F160E6B6FDF0E6A6FFF
:101D0000160E6D6F800E6C6F160E6F6F240E6E6F59
:101D1000150E716FC80E706F150E736F6E0E726FA9
:101D2000150E756F160E746F140E776FBF0E766FEB
:101D3000140E796F690E786F140E7B6F150E7A6F23
:101D4000130E7D6FC20E7C6F130E7F6F710E7E6F50
:101D5000130E816F210E806F120E836FD20E826F71
:101D6000120E856F840E846F120E876F380E866F89
:101D7000110E896FED0E886F110E8B6FA30E8A6F97
:101D8000110E8D6F5A0E8C6F110E8F6F120E8E6F9B
:101D9000100E916FCC0E906F100E936F870E926F96
:101DA000100E956F420E946F0F0E976F9669996F94
:101DB000BD0E986F0F0E9B6F7C0E9A6F0F0E9D6F6E
:101DC0003D0E9C6F0E0E9F6FFE0E9E6F0E0EA16F4E
:101DD000C00EA06F0E0EA36F830EA26F0E0EA56F26
:101DE000470EA46F0E0EA76F0C0EA66F0D0EA96FF7
:101DF000D20EA86F0D0EAB6F990EAA6F0D0EAD6FC0
:101E0000610EAC6F0D0EAF6F2A0EAE6F0C0EB16F80
:101E1000F40EB06F0C0EB36FBE0EB26F0C0EB56F3A
:101E20008A0EB46F0C0EB76F560EB66F0C0EB96FEC
:101E3000230EB86F0B0EBB6FF10EBA6F0B0EBD6F9A
:101E4000C00EBC6F000112000101C16B340EC06FE7
:101E5000020E1A6E0001800E1A5C36E21A04066E3B
:101E600001EEBEF0D8900634E926000EEA22EECF4D
:101E700004F0EFCF05F004C00CF005C00DF006EC47
:101E800001F00FC013F00EC012F00DC011F00CC025
:101E900010F0330E0F6E0E6E030E0D6E840E0C6E70
:101EA00025EC00F0B3EC00F0006E0DC001F001EE87
:101EB000BEF0D8901A34E926000EEA2200C0EEFFE8
:101EC00001C0EFFF1A2AC6E312000101C16B2F0EF9
:101ED000C06F020E1A6E0001800E1A5C20E21A0416
:101EE000066E01EEBEF0D8900634E926000EEA2216
:101EF000EECF04F0EFCF05F0140E0424006E000EB8
:101F00000520016E01EEBEF0D8901A34E926000ECD
:101F1000EA2200C0EEFF01C0EFFF1A2ADCE3120044
:101F20000101C16B2E0EC06F020E1A6E0001800EF1
:101F30001A5C37E21A04066E01EEBEF0D890063441
:101F4000E926000EEA22EECF04F0EFCF05F004C040
:101F50000CF005C00DF006EC01F00FC013F00EC040
:101F600012F00DC011F00CC010F00A0E0F6ED70E5B
:101F70000E6E470E0D6E820E0C6E25EC00F0B3EC6B
:101F800000F0006E0DC001F001EEBEF0D8901A34E2
:101F9000E926000EEA2200C0EEFF01C0EFFF1A2A78
:061FA000C5E31200FFD7AB
:020000040030CA
:0300010006160ED2
:020005008580F4
:060008000FC00FE00F40E5
:00000001FF
